S107000002010032C3
S104000B32BE
S104001332B6
S104001B32AE
S104002332A6
S1130100758780758922758DFF758BFFD28E7598E2
S1130110427930782C770009D8FB7930782C889094
S1130120B700FB09D8F87590FF79307E297C0078F8
S113013000313C78147C00313C0201297D16ECF539
S1130140904390F0D392B5EC54F07003C392B50091
S11301500000B80005A2B002015EA2B2B2B3501E04
S1130160E744006034E590F454F0232323234480CF
S113017031A2EE31A2740031A27700020199E74462
S1130180007016E590F454F023232323449031A205
S1130190EE31A2744631A27701090E0CDD01220270
S10D01A0013E3099FDC299F5992241
S9030000FC
